:1000000018C1000032C1000030C100002EC1000044
:100010002CC100002AC1000028C1000026C1000038
:1000200024C1000022C1000020C100000C942A104D
:100030001CC10000AEC1000018C10000ABC7000029
:1000400014C1000012C1000010C100000EC1000068
:100050000CC100000AC1000008C1000006C1000078
:1000600004C1000002C1000000C10000FEC0000089
:10007000FCC0000012011001FF000010EB0304217E
:1000800000020102030109022000010100C032093F
:1000900004000002FF0000000705820240000A077A
:1000A00005020240000A040309040C034100540045
:1000B0004D0045004C00000018034100560052005E
:1000C00049005300500020006D006B0049004900BA
:1000D00000001C03300030003000320030003000DF
:1000E00030003100320033003400350000000000E1
:1000F00009000A000A000B000C000D000D000E00A4
:100100000F0010001000120013001300140016005E
:100110001600180019001A001C001D001F00200006
:10012000220023002500270029002B002E0030008C
:100130003200340037003A003D00400043004600E2
:100140004A004E00520055005A005E0063006800ED
:100150006D00730078007E0084008B009100990090
:10016000A000A900B100B900C300CC00D600E10096
:10017000EC00F700040111011E012D013B014B01B0
:100180005B016C017D019101A501BA01CF01E6017E
:10019000FE01160231024C026A028802A802CA025B
:1001A000ED021103380360038B03B803E70318045F
:1001B0004B048104B904F50434057505B90501063D
:1001C0004E069D06EF064807A30704086508D008F9
:1001D0004009B6092B0AAB0A300BC30B510CEE0CCD
:1001E0008F0D400EF60EAF0F681047111412F51266
:1001F000ED13E214F015F9161B185C19911AE51BA2
:10020000251D831E0320AB21302332250F27F12823
:10021000F82A1A2D492FA1311434A1364539173C3B
:100220001A3F34426045DF48704C40004101424370
:10023000030011241FBECFEFD2E0DEBFCDBF11E01F
:10024000A0E0B1E0E8EAF6E202C005900D92A23427
:10025000B107D9F711E0A2E4B1E001C01D92A535C4
:10026000B107E1F74ED00C945213CACE85B18F710D
:10027000806C85B9089585B18F71806485B90895C2
:100280008EB3843089F4CAD182E08093E9008091F2
:10029000E80082FF09C085B18F71806C85B98FD06D
:1002A00085B18F71806885B9089582E060E842E386
:1002B0000E94840F80FD02C090E401C090E885B1E7
:1002C0008F71982B95B9089584B7877F84BF88E193
:1002D0000FB6F89480936000109260000FBE80E02B
:1002E00090E020E80FB6F8942093610080936100BD
:1002F0000FBE84B1806E84B985B18F7185B90C94BD
:100300001B10E2DF89D185B18F71806485B9789443
:10031000489902C090E201C090E085B18F7D982B92
:1003200095B9AEDF0E942613F3CFDA01292F3327C8
:10033000223049F0233061F0213021F5E4E7F0E08C
:1003400082E190E023C0E6E8F0E080E290E01EC0A9
:10035000813059F0813028F0823059F0833091F4A7
:100360000CC0E6EAF0E084910BC0EAEAF0E0849188
:1003700007C0E8EBF0E0849103C0E2EDF0E0849187
:1003800090E004C0E0E0F0E080E090E0ED93FC93CA
:1003900008951F920F920FB60F9211248F9381E050
:1003A0008ABD88E10FB6F8948093600010926000D7
:1003B0000FBE8F910F900FBE0F901F901895FF9258
:1003C0000F931F931091F1001ABC8EE028E130E0EA
:1003D0000FB6F894A895209360000FBE809360003C
:1003E00080916000806480936000143109F4CBC078
:1003F000153110F51A3009F4ADC01B3068F4143013
:1004000038F4123008F054C0113009F0D4C033C0B1
:10041000163009F0D0C078C0113109F4AFC01231E4
:1004200020F4103109F0C7C0A7C0123109F4AEC0E2
:10043000133109F0C0C0A4C0193109F4ACC01A319D
:1004400068F4163109F49FC0163108F499C01731C9
:1004500009F4A1C0183109F0AEC09AC01D3109F4E9
:100460009DC01D3108F494C0103509F49BC01135AE
:1004700009F0A1C095C08091E8008B778093E800D7
:1004800082E08093E9008091EC0081608093EC0031
:100490001093F1001092F1008AE08093F10080E067
:1004A00091E06AE070E040E050E00E94C81199C01D
:1004B0000091F100123011F0FF2402C0F090F10021
:1004C0008091E8008B778093E80082E08093E900D8
:1004D0008091EC0081608093EC001093F100802FFC
:1004E000B6D0123041F481FF0DC01092F100802F80
:1004F0006F2DB5D076C080FF05C01092F100802F1F
:100500009ED06DC080EC6BC086E491E064E070E04A
:1005100040E050E00E9429118091E8008B778093A1
:10052000E80082E08093E9008091EC008160809394
:10053000EC008091460190914701A0914801B09153
:100540004901B7FF03C081E08093450186E08093B5
:10055000F1000FC08091E8008B778093E80082E083
:100560008093E9008091EC0081608093EC0010930F
:10057000F1001092F10035C071D438C03BD436C0C0
:10058000812FF6D233C0812F42D230C0F1D12EC09C
:10059000812FE6D02BC0812F9DD028C04CD126C002
:1005A00037D624C085D722C08091E8008B7780930E
:1005B000E8000E94B60F8091F2008034A9F3809188
:1005C000E8008B778093E80082E08093E9008091D7
:1005D000EC0081608093EC001093F10089EC809333
:1005E000F1008091E8008E778093E80088E10FB6F3
:1005F000F89480936000109260000FBE0E94B60FC6
:1006000082E08093E9008091EC008E7F8093EC0083
:100610001F910F91FF90089535D0ECC40895982F45
:10062000EBE0F1E08081981741F081E0E632F807D5
:1006300011F03396F7CFE0E0F0E0CF010895EFDF5F
:10064000FC01009711F480E0089582810895E7DFAE
:10065000FC01009711F480E00895818108950F93C3
:100660001F93182F062FDBDFFC01009741F0028358
:100670001E3929F480E090E0602F0E9440131F9102
:100680000F9108950F931F938EE9C9DF8C0180E0CD
:1006900090E00E943813F80182831F910F91089512
:1006A000282F40EA5FE003C0CA010197F1F7222337
:1006B00021F08AB521508823B9F30895982F8091AD
:1006C0002901882329F09EBD0DB407FEFDCF0895B2
:1006D000892FD0C4DF92EF92FF920F931F93DF9385
:1006E000CF9300D000D0CDB7DEB7D82E8E010F5FEC
:1006F0001F4FC80164E070E040E050E00E947B11B1
:100700008091E8008B778093E80082E08093E90095
:100710008091EC0081608093EC0085E0E82EF12C64
:10072000EC0EFD1EF80181918F01C8DF0E151F052B
:10073000C9F7D092F1001092F1001092F10080916F
:10074000E8008E778093E8000F900F900F900F9045
:10075000CF91DF911F910F91FF90EF90DF9008955F
:10076000BF92CF92DF92EF92FF920F931F93DF938E
:10077000CF93CDB7DEB729970FB6F894DEBF0FBE83
:10078000CDBFB82ECE01059665E070E040E050E0A8
:100790000E947B118091E8008B778093E80082E0D3
:1007A0008093E9008091EC0081608093EC008E01E1
:1007B0000A5F1F4F7E010894E11CF11C9AE0C92ECC
:1007C000D12CCC0EDD1EF801908180912901882367
:1007D00031F09EBD0DB407FEFDCF8EB502C0892F4E
:1007E00049D4F70181937F010F5F1F4F0C151D0541
:1007F00051F7B092F1001092F1008D81FE01E80FE7
:10080000F11D80818093F1001092F1008091E80049
:100810008E778093E80029960FB6F894DEBF0FBE5E
:10082000CDBFCF91DF911F910F91FF90EF90DF909F
:10083000CF90BF900895EF92FF920F931F93DF9395
:10084000CF93CDB7DEB7C250D1400FB6F894DEBF1C
:100850000FBECDBFCE01019663E070E040E050E0F6
:100860000E947B1134E0E32EF12CEC0EFD1E698119
:1008700070E0C70140E050E00E947B118091E800E9
:100880008B778093E80082E08093E9008091EC0010
:1008900081608093EC008DE18093F1001092F10073
:1008A00000E00BC08981081728F4F701E00FF11D63
:1008B000808101C080E002DF0F5F8B81081790F319
:1008C00010E024E0E22EF12CEC0EFD1E2CC08981FC
:1008D00090912901081778F4F701E00FF11D80814C
:1008E000992331F08EBD0DB407FEFDCF8EB501C04A
:1008F000C1D30F5F0AC0992331F01EBC0DB407FEAF
:10090000FDCF8EB502C080E0B5D38093F100809119
:10091000E80085FD07C08091E8008E778093E800AD
:100920000E94B60F1F5F8A81181788F21092F1009B
:100930009091E8008091E8008E778093E80095FD23
:1009400009C00E94B60F8091E8008E778093E8007E
:100950000E94B60FCE5FDE4F0FB6F894DEBF0FBE1B
:10096000CDBFCF91DF911F910F91FF90EF90089530
:10097000EF92FF920F931F93DF93CF9300D000D09D
:1009800000D0CDB7DEB7CE01019666E070E040E062
:1009900050E00E947B118091E8008B778093E80003
:1009A00082E08093E9008091EC0081608093EC000C
:1009B0008E010D5F1F4F47E0E42EF12CEC0EFD1E63
:1009C000F80181918F017ADE0E151F05C9F78A8122
:1009D000882321F4898164DE90E002C076D3982FC9
:1009E00082E18093F1009093F1008091E8008E778E
:1009F0008093E80026960FB6F894DEBF0FBECDBFF9
:100A0000CF91DF911F910F91FF90EF900895DF92AA
:100A1000EF92FF920F931F93DF93CF9300D00F922B
:100A2000CDB7DEB7F82ECE01019663E070E040E06E
:100A300050E00E947B1189819A81282F892F922F63
:100A40009A8389838091E8008B778093E80082E025
:100A50008093E9008091EC0081608093EC00F0923B
:100A6000F1001092F10000E010E068E0D62EEE24D4
:100A7000E39459C080914501882319F041D3109225
:100A800045018B811BDE8091460190914701A09129
:100A90004801B0914901892F9A2FAB2FBB270EDE59
:100AA000809146010BDE80912901882331F01EBC24
:100AB0000DB407FEFDCF8EB502C080E0DBD280937F
:100AC000F1008091E80085FD07C08091E8008E77F5
:100AD0008093E8000E94B60F24E1F21619F48B818E
:100AE0008D258B8300FD03C086E1F816D1F480913B
:100AF000460190914701A0914801B09149010196AA
:100B0000A11DB11D8093460190934701A093480118
:100B1000B093490126E1F21621F0892B11F4E092FD
:100B200045010F5F1F4F89819A810817190708F443
:100B3000A1CF1092F1009091E8008091E8008E77AB
:100B40008093E80095FD09C00E94B60F8091E800EF
:100B50008E778093E8000E94B60F0F900F900F9051
:100B6000CF91DF911F910F91FF90EF90DF9008954B
:100B70002F923F924F925F926F927F928F929F92AD
:100B8000AF92BF92CF92DF92EF92FF920F931F939B
:100B9000DF93CF93CDB7DEB7C950D1400FB6F894ED
:100BA000DEBF0FBECDBF982ECE01019669E070E08A
:100BB00040E050E00E947B1169817A81862F672F87
:100BC000782F21E06130720798F08091E8008B77F0
:100BD0008093E80082E08093E9008091EC008160DE
:100BE0008093EC009092F10080EC8093F100E3C0E0
:100BF0007A836983CE010A9640E050E00E947B111F
:100C000089819A810A968F739070892B39F480912B
:100C1000E8008B778093E8000E94B60F8091E8008F
:100C20008B778093E80082E08093E9008091EC006C
:100C300081608093EC0083E1981611F4888401C0F0
:100C4000898440904601509047016090480170901F
:100C50004901EE24FF24AAE0AA2EB12CAC0EBD1E41
:100C6000CC24DD24F8E02F2E3324339471C0F50119
:100C700010810B8180914501882319F041D2109297
:100C800045018D811BDD8091460190914701A09126
:100C90004801B0914901892F9A2FAB2FBB270EDD58
:100CA000809146010BDD812F09DDF3E19F1619F4D8
:100CB0008D8182258D83E114F10489F4181579F072
:100CC000C0FE06C023E1921619F48F81886002C02D
:100CD0008F81877F8F83E0904601F090470100FD70
:100CE00012C0E114F10421F403FD02C0097F026087
:100CF000802FB701482D2C810F810BD2282F8823FC
:100D000071F5EE24FF24C0FC03C085E19816D1F4F0
:100D10008091460190914701A0914801B09149010D
:100D20000196A11DB11D8093460190934701A093A8
:100D30004801B0934901E3E19E1621F4892B11F497
:100D4000309245010894A11CB11C0894C11CD11C0F
:100D500089819A81C816D90608F489CF20E08B8151
:100D600087FF25C08E81AADC852D9927A7DC842DDD
:100D7000A5DC80E0A3DC8B8185FF06C0E114F104D3
:100D800019F48F7C80618B838B81B701482D2C8176
:100D90000F81BFD1282FF3E19F1649F480914601BE
:100DA00090914701892B19F481E08093450190923D
:100DB000F1002093F1008091E8008E778093E800A5
:100DC000C75FDE4F0FB6F894DEBF0FBECDBFCF9129
:100DD000DF911F910F91FF90EF90DF90CF90BF9028
:100DE000AF909F908F907F906F905F904F903F90CB
:100DF0002F9008950F931F93DF93CF9300D0CDB71B
:100E0000DEB7CE01019662E070E040E050E00E9463
:100E10007B1108EE10E0F80180818B77808382E0FF
:100E20008093E900ECEEF0E080818160808389812D
:100E300037DC80E0B7D1F2D08A8132DCE1EFF0E03C
:100E400081E180831082F80180818E7780830F900A
:100E50000F90CF91DF911F910F9108958F929F92E4
:100E6000AF92BF92CF92DF92EF92FF920F931F93B8
:100E7000DF93CF93CDB7DEB72F970FB6F894DEBFD1
:100E80000FBECDBFCE0105966BE070E040E050E0B4
:100E90000E947B118091E8008B778093E80082E0CC
:100EA0008093E9008091EC0081608093EC001092C7
:100EB00046011092470110924801109249018F811A
:100EC000EFDB7CD181E06ED18E81EADB1CE0812EEC
:100ED000912C8C0E9D1E5E010894A11CB11CB0E1EA
:100EE000CB2ED12CCC0EDD1E2AC08985D9DBF80192
:100EF000908180912901882331F09EBD0DB407FEB9
:100F0000FDCF8EB502C0892FB5D0F70181937F0147
:100F10000F5F1F4F0C151D0541F78B858823D1F0FE
:100F2000FE01E80FF11D90818A85981799F080E005
:100F300039D18E81B5DB81E035D18E81B1DB9885E9
:100F4000992351F08AB5882339F491509887840108
:100F50007501CBCF90E001C090EC80E18093F1006F
:100F60009093F1008091E8008E778093E8002F96AF
:100F70000FB6F894DEBF0FBECDBFCF91DF911F91AA
:100F80000F91FF90EF90DF90CF90BF90AF909F9028
:100F90008F9008951F920F920FB60F9211248F9386
:100FA000199908C08091420187FF02C02A9A1BC08C
:100FB0002A9819C080914201880F80934201809144
:100FC000430181508093430180914301882321F4A0
:100FD0001092810082E086BB1B9B05C0809142017C
:100FE000816080934201199A8F910F900FBE0F90EC
:100FF0001F9018953E9A10926F00109285001092E3
:10100000840081E090E0909389008093880080E4E0
:101010008093800089E08093810008958091290168
:10102000882349F084B1897F84B985B1867F85B9E9
:101030001CBC1DBC089584B1897F84B985B1867FAD
:1010400085B9D8CF92E090936F00109285001092EE
:101050008400E82FF0E0EE0FFF1FEE51FF4F859167
:101060009491909389008093880010928000109250
:10107000810008958093420188E08093430180912C
:10108000420187FF02C02A9A01C02A981092850067
:10109000109284008AE0809381008091430188232C
:1010A00019F08AB58823C9F310928100809142011A
:1010B0000895982F80912901882329F09EBD0DB4B1
:1010C00007FEFDCF0895892FD5CF80EFF2DF80E0B6
:1010D000F0DF80E0EEDF80912901882331F01EBC33
:1010E0000DB407FEFDCF8EB502C080E0C3DF80FFE8
:1010F00003C08AB5882349F38AB5811181E8089530
:101100008DE4D7DF80E0D5DF80914801D2DF80E039
:10111000D0CFFF920F931F93CF93DF93EB01F42E69
:1011200090E08E778830910599F18930910534F4FB
:101130008230910559F0049769F50BC08032910512
:1011400041F08034910521F1409721F5822FA8DAF2
:1011500021C08D2F9927182F802FABDF812FA9DF7A
:101160008C2FA7DF80912901882331F01EBC0DB49C
:1011700007FEFDCF8EB502C080E07CDF8F1519F42D
:101180008AB5882349F38AB5882321F080E803C013
:101190009CDF01C080E0A895DF91CF911F910F9156
:1011A000FF900895882339F0249A8EE948DA88233D
:1011B00019F42C9A089524982C98089588E93FDA18
:1011C000E82F8730D8F481E080932901F0E0E65DD4
:1011D000FD4FE491E061209A289A84B1866084B939
:1011E00023982B9AE6FF03C08DB5816002C08DB5B0
:1011F0008E7F8DBD2098E064ECBD0895109229018A
:1012000084B1866084B985B1896085B98E2F1ACF83
:10121000DF93CF930F92CDB7DEB7CE01019661E099
:1012200070E040E050E00E947B118091E8008B77F5
:101230008093E80082E08093E9008091EC00816077
:101240008093EC0099819093440181E58093F100B3
:10125000913011F480EC01C080E08093F100809126
:10126000E8008E778093E8000F90CF91DF9108958A
:101270009B01AC01652F922F272F782F822F089585
:10128000AF92BF92CF92DF92EF92FF920F931F9394
:10129000DF93CF93CDB7DEB7C850D1400FB6F894E7
:1012A000DEBF0FBECDBFCE01019668E070E040E02A
:1012B00050E00E947B116B817C818D819E810F812A
:1012C0001885202F012F122F18870F83D1DF6B83F2
:1012D0007C838D839E83CE010996B80140E050E067
:1012E0000E947B118F81988509968F739070892B4E
:1012F00031F48091E8008B778093E80037D68091B5
:10130000E8008B778093E80082E08093E900809189
:10131000EC0081608093EC0080914401882379F592
:1013200089818330A9F0843028F4813069F08230DB
:10133000A9F40CC0853031F0853008F44CC08630FB
:1013400069F40AC088E048C044E209C04CE207C022
:1013500045E383E366E305C04AE101C04EE283E270
:1013600066E2EB80FC800D811E81AF80B8842A810B
:1013700099E0C92ED12CCC0EDD1E01D308C04F81BF
:1013800058858B819C81BE01675F7F4F04D5882380
:1013900011F090E001C093E080E58093F10084E0DB
:1013A0008093F1009093F1008091E8008E77809314
:1013B000E800C85FDE4F0FB6F894DEBF0FBECDBFAA
:1013C000CF91DF911F910F91FF90EF90DF90CF9021
:1013D000BF90AF9008958CE44B815C816D817E81DC
:1013E000298534D3D4CFDF93CF93CDB7DEB7C750A1
:1013F000D1400FB6F894DEBF0FBECDBFCE0101962F
:1014000067E070E040E050E076D76A817B818C81B4
:101410009D812EDFAB01BC014A835B836C837D839E
:101420002E813F81822F232F382F3F832E8380915F
:10143000E8008B778093E80082E08093E900809158
:10144000EC0081608093EC0080914401FE013896AD
:10145000882329F4CB01BA01AF011AD304C0CA0111
:10146000BF01A901D0D4882311F493E001C090E01A
:1014700080E58093F10085E08093F1009093F10086
:10148000992339F46E817F81CE01089640E050E0C7
:101490007FD78091E8008E778093E800C95FDE4FA8
:1014A0000FB6F894DEBF0FBECDBFCF91DF91089588
:1014B000DF93CF93CDB7DEB729970FB6F894DEBF91
:1014C0000FBECDBF9091F100943009F4AEC09530BD
:1014D00048F4923091F1933008F04BC0913009F00C
:1014E0004AC10AC0963009F4A4C0963008F49FC0DF
:1014F000973009F040C1E5C08091E8008B77809378
:10150000E80082E08093E9008091EC0081608093A4
:10151000EC0080914401882311F4B3D305C08230DC
:1015200011F090E002C0B6D4982F80E58093F100CE
:1015300081E08093F1008927C1C08091E8008B771A
:101540008093E8009093E9008091EC0081608093A3
:10155000EC0080914401882311F488D301C08FD41A
:1015600080E58093F10082E08093F1001092F10019
:10157000FDC0CE01059665E070E040E050E0BBD6CE
:101580006E817F818885998573DEAB01BC014E83B6
:101590005F83688779878091E8008B778093E80084
:1015A00082E08093E9008091EC0081608093EC0000
:1015B000809144012D81882339F52430C1F02530F4
:1015C00038F4223071F0233080F42130D1F40BC094
:1015D000263089F0263068F0273079F0283089F4F9
:1015E0000EC080E20FC080E40DC088E60BC080E32F
:1015F00009C082E207C08AE205C082E303C088E135
:1016000001C080E090D207C0213011F084E101C018
:1016100080E1BA01A5D3882311F090E001C093E0E6
:1016200080E58093F10083E09DC02ADEA4C0DBDE6C
:10163000A2C0CE01059661E070E040E050E05BD6CC
:101640008091E8008B778093E80082E08093E90046
:101650008091EC0081608093EC00809144018823AC
:1016600011F091E013C08D81813021F0823021F49E
:1016700089E303C088E301C088E7BE016F5F7F4F45
:10168000BFD2882311F493E001C090E080E58093FD
:10169000F10086E08093F1009093F100992309F026
:1016A00065C089819A81AB81BC819D014427552702
:1016B0002093F1008093F100892F99278093F10006
:1016C00055C08091F100833069F1843028F4813075
:1016D00049F0823029F41BC0843049F1853061F132
:1016E00091E02FC02091F100B22F2091F100A22FA4
:1016F0002091F100922F2091F100822F80932A01F6
:1017000090932B01A0932C01B0932D0119C08091CF
:10171000F100382F8091F100282F30932F01209372
:101720002E010EC08091F1008093300109C080919C
:10173000F1008093310104C08091F1008091F100AB
:1017400090E08091E8008B778093E80082E08093BE
:10175000E9008091EC0081608093EC0080E580934B
:10176000F10087E08093F1009093F1008091E80010
:101770008E778093E80029960FB6F894DEBF0FBEEF
:10178000CDBFCF91DF9108954D99FECF4D9BFECFF8
:101790004D99FECF5B9A539A8091C9008F7E8093BA
:1017A000C9008091C90088608093C90081E080935E
:1017B0004A01089580914A01882309F4E5DF80E019
:1017C0004D99FECF4D9BFECF4D99FECF8F5F8C3054
:1017D000B9F7089510924A01249A2C9885E08A95C9
:1017E000F1F78AB188628AB952988FE190E09093BC
:1017F000CD008093CC0088E08093C9008FE6809371
:10180000CA00D8DFD7CF10924A018AB188628AB95C
:1018100052985B9A85E08A95F1F78FE190E090937A
:10182000CD008093CC0088E08093C9008FE6809340
:10183000CA00C0DFBFCF1F93182F80914A018823B1
:1018400009F4A2DF8091C80085FFFCCF8091C80019
:1018500080648093C8001093CE001F9108958091FA
:10186000C80086FFFCCF8091C80080648093C800C8
:101870008091C900877F8093C9008091C9008061F1
:101880008093C90053985B9810924A010895809103
:101890004A01882309F0E3DF8091C80087FD03C077
:1018A0008AB58823C9F38091CE00089580914A01BA
:1018B000882309F0D4DF8091C800806C8093C80031
:1018C0001092C9001092CA008AB1877D8AB98BB183
:1018D000837D8BB924982C98089580914A018823A0
:1018E00009F0BDDF80EC8093C8001092C90010920F
:1018F000CA008AB1877D8AB98BB1837D8BB908957F
:10190000EF92FF920F931F937B018C01862F93DF41
:10191000BB27A12F902F8F2D8EDFC801AA27BB27B1
:101920008ADFE12EFF24002711278E2D84DF1F91EF
:101930000F91FF90EF90089590E0A0E0B0E020912B
:101940002A0130912B0140912C0150912D01822BC5
:10195000932BA42BB52BBC01CD01D2CF8BE66BDF33
:101960008FE0EADF80E267DF92DF982F8AB5882375
:1019700011F080E0089597FDF5CF81E008957F9202
:101980008F929F92AF92BF92CF92DF92EF92FF928F
:101990000F931F93CF93DF93882E962E742EE6011C
:1019A000C22E20FF10C0DADF882309F440C08CE487
:1019B00042DF8AE0C1DF892D3EDF8CE43CDF8BE033
:1019C000BBDF81E038DFA114B104E9F0C7DF882371
:1019D00071F18CE430DF8AE0AFDF882D2CDF8BE6FD
:1019E0002ADFC801B7018CDF80EA25DF8A2D81500C
:1019F00022DF84E620DF89911EDF0894A108B10868
:101A0000A114B104C1F7C1FE10C0A8DF882379F08A
:101A10008CE411DF8AE090DF872D0DDF8CE40BDF93
:101A2000C801B7016DDF80E006DF81E001C080E022
:101A3000DF91CF911F910F91FF90EF90DF90CF90AA
:101A4000BF90AF909F908F907F900895CF92DF923C
:101A5000EF92FF920F931F93D82E7A018B01C22E23
:101A60007DDF882371F08CE4E6DE8AE065DF8D2D72
:101A7000E2DE8CE4E0DEC801B70142DF8C2DDBDE64
:101A800081E01F910F91FF90EF90DF90CF9008952C
:101A9000CF92DF92EF92FF920F931F93CF93DF933A
:101AA0007B018C016A01E90159DF882311F490E080
:101AB00023C08CE4C0DE8AE03FDF83E4BCDE8BE63B
:101AC000BADEC801B7011CDF80EAB5DE9E012150F5
:101AD000822FB1DE84E2AFDE04C0D9DEF60181934D
:101AE0006F01209721F08AB521978823B1F38AB539
:101AF00090E0882309F491E0892FDF91CF911F9125
:101B00000F91FF90EF90DF90CF90089580E893DEE3
:101B1000BEDE982F8AB5882311F080E0089591FFEA
:101B2000F5CF81E00895CF92DF92EF92FF921F935D
:101B3000182F6A017B0112DF882309F45AC0103480
:101B400031F48CE478DE8AE0F7DE80E439C01033CB
:101B500009F03DC08CE46FDE8AE0EEDE86E36BDEEA
:101B60008CE469DE8BE0E8DE81E065DEF7DE882369
:101B700009F43FC08CE45FDE8AE0DEDE83E35BDEF7
:101B80008BE659DEC701B601BBDE80EA54DE8091E8
:101B90002E01815050DE84E64EDE10E003C080E06E
:101BA0004ADE1F5F212F30E080912E0190912F019E
:101BB00028173907A0F38CE43EDE8AE0BDDE80E31F
:101BC0003ADE8CE438DE8BE0B7DE81E00CC08CE4DA
:101BD00032DE8AE0B1DE812F2EDE8CE42CDEC701FE
:101BE000B6018EDE80E027DE91DF882319F081E0E8
:101BF00001C080E01F91FF90EF90DF90CF9008959B
:101C00001F93CF93DF93182FEB01A8DE882341F1B8
:101C10008CE411DE8AE090DE812F0DDE8CE40BDE99
:101C20008BE08ADE81E007DE71DF8823C9F096DE73
:101C30008823B1F08BE6FFDD84E07EDE80EAFBDD09
:101C400082E0F9DD84E2F7DD22DE888320DE89830D
:101C50001EDE8A838AB590E0882319F491E001C0E2
:101C600090E0892FDF91CF911F9108954FDF81EC94
:101C7000E2DD80E0E0DD81E8DEDD09DE8823B9F722
:101C80002CCEEF92FF920F931F93DF93CF93CDB79C
:101C9000DEB728970FB6F894DEBF0FBECDBFB3DD19
:101CA00081ECC9DD89E5C7DD82ECC5DD82E0C3DDFD
:101CB00080EEC1DD8E01085F1F4F7E010894E11C9C
:101CC000F11CD701E2E3F1E088E001900D92815030
:101CD000E1F7F8018081AFDD015010400C171D07BE
:101CE00081F714DF28960FB6F894DEBF0FBECDBF84
:101CF000CF91DF911F910F91FF90EF900895282FC2
:101D00008F70806930E020733070220F331F822B78
:101D100092CD0F931F938C0188E68DDD802F8BDD94
:101D200089E689DD012F1127802F85DD1F910F9115
:101D3000089520913101822F8F70806130E02073EF
:101D40003070220F331F822B76DDA1DD982F8AB5EC
:101D5000882311F080E0089597FDEBCF81E008958E
:101D60001F93CF93DF93182FEB01E3DF882379F0E4
:101D700080913001C4DF812F5EDDCE018160C9DF3B
:101D800080E659DD80E057DDD4DF811181E0DF910D
:101D9000CF911F910895EF92FF920F931F93CF93CE
:101DA000DF937C018B01EA01C4DF882321F1C0FFAE
:101DB00006C0F801EC0FFD1F8FEF80832196809104
:101DC00030019DDF8DE137DDC701A3DF10C0B1DF3A
:101DD000882389F084E62FDDF80180812CDD84E6FC
:101DE0002ADDF80181810E5F1F4F25DD22972097A4
:101DF00071F781E001C080E0DF91CF911F910F91D9
:101E0000FF90EF900895EF92FF920F931F93CF935F
:101E1000DF938C017B01EA018CDF882311F490E0D1
:101E200019C0809130016BDF80E005DDC80171DFF2
:101E300006C084E200DD2BDDF70181937F0120974E
:101E400021F08AB521978823A1F38AB590E08823F1
:101E500009F491E0892FDF91CF911F910F91FF90AD
:101E6000EF90089580E8E7DC12DD982F8AB588238B
:101E700011F080E0089591FFF5CF81E00895F2DF41
:101E800080ECD9DC80E0D7DC81E8D5DC00DD88237C
:101E9000B9F70CCDEF92FF920F931F93DF93CF937F
:101EA000CDB7DEB728970FB6F894DEBF0FBECDBF13
:101EB00091DC82ECC0DC82E0BEDC80EEBCDC8E011A
:101EC000085F1F4F7E010894E11CF11CD701EAE373
:101ED000F1E088E001900D928150E1F7F8018081F6
:101EE000AADC015010400C171D0781F7BBDF2896B4
:101EF0000FB6F894DEBF0FBECDBFCF91DF911F911B
:101F00000F91FF90EF9008958093E9008091EB008E
:101F100081608093EB001092ED006093EC004093A1
:101F2000ED008091EE00881F8827881F089580911A
:101F30004D0188238CF403C08EB38823B1F08091C7
:101F4000E80082FFF9CF8091E8008B778093E8006A
:101F500008958EB3882349F08091E80080FFF9CF7F
:101F60008091E8008E778093E80008954091E40026
:101F70005091E50024E68091EC0080FF23C0809121
:101F8000E80080FD1DC08EB3882311F482E008951F
:101F9000853011F483E008958091EB0085FF02C045
:101FA00081E008958091E4009091E5008417950701
:101FB00011F3222311F484E008952150AC01DBCF0A
:101FC00080E008958091E80082FFDDCFF9CF3CD01A
:101FD0003ED08091D8008F778093D8008091D80030
:101FE00080688093D8008091D8008F7D8093D8003E
:101FF00084E089BD86E089BD09B400FEFDCF1EBA2C
:1020000010924B0180E060E042E17EDF8091E100D0
:102010008E7F8093E1008091E20081608093E200F6
:102020008091E20088608093E2008091E0008E7FE2
:102030008093E0000895E3E6F0E080818E7F808366
:1020400081E080934C01C3CF1092E200089510927A
:10205000E10008951F920F920FB60F9211242F9353
:102060003F934F935F936F937F938F939F93AF9320
:10207000BF93EF93FF938091E10082FF0AC08091AC
:10208000E20082FF06C08091E1008B7F8093E10037
:10209000DCD28091E10080FF17C08091E20080FFD8
:1020A00013C08091E2008E7F8093E2008091E20075
:1020B00080618093E2008091D80080628093D80094
:1020C00019BC1EBA0E943B018091E10084FF2DC023
:1020D0008091E20084FF29C084E089BD86E089BD4B
:1020E00009B400FEFDCF8091D8008F7D8093D80089
:1020F0008091E1008F7E8093E1008091E2008F7EED
:102100008093E2008091E20081608093E200809100
:102110004B01882331F48091E30087FD02C081E008
:1021200001C084E08EBB0E9436018091E10083FFF4
:1021300021C08091E20083FF1DC08091E100877F74
:102140008093E10082E08EBB10924B018091E10010
:102150008E7F8093E1008091E2008E7F8093E20089
:102160008091E20080618093E20080E060E042E1E3
:10217000CBDE6BD2FF91EF91BF91AF919F918F9189
:102180007F916F915F914F913F912F910F900FBE73
:102190000F901F901895FC014091530150915401EC
:1021A0004617570710F490E03FC06115710511F014
:1021B000AB01F9CF8091E8008E778093E80040E092
:1021C00050E0F1CF8EB3882309F43FC0853009F485
:1021D0003EC08091E80083FF02C081E008958091B5
:1021E000E80082FD2CC08091E80080FF1DC0809136
:1021F000F200282F30E008C084918093F1003196DE
:10220000415050402F5F3F4F4115510519F020318B
:10221000310590F390E02031310509F491E080918F
:10222000E8008E778093E8004115510559F699230F
:1022300049F605C08EB3882341F0853041F0809186
:10224000E80082FFF7CF80E0089582E0089583E000
:102250000895BF92CF92DF92EF92FF920F931F9358
:10226000CF93DF938C01EB016A0180DEB82E8823C7
:10227000B9F521970C0F1D1F2196C114D10439F017
:10228000F60180819181C81BD90B081B190BEE2424
:10229000FF2424C08091E80085FD16C08091E800ED
:1022A0008B778093E800D2D1C114D10449F0F601B4
:1022B000808191818E0D9F1D9183808385E011C067
:1022C00055DE882359F00DC08091F100F80180831C
:1022D0000150104021970894E11CF11C2097D1F681
:1022E0008B2DDF91CF911F910F91FF90EF90DF9099
:1022F000CF90BF900895BF92CF92DF92EF92FF925E
:102300000F931F93CF93DF93EC018B017A012EDEA5
:10231000B82E882391F5E114F10439F0F70180819A
:102320009181081B190BC80FD91FCC24DD2422C0B2
:102330008091E80085FD16C08091E8008B7780933E
:10234000E80084D1E114F10449F0F7018081918122
:102350008C0D9D1D9183808385E010C007DE88234E
:1023600049F00CC08091F10089930150104008940D
:10237000C11CD11C01151105D9F68B2DDF91CF9110
:102380001F910F91FF90EF90DF90CF90BF90089535
:10239000BF92CF92DF92EF92FF920F931F93CF9352
:1023A000DF93EC018B017A01E1DDB82E882391F5F2
:1023B000E114F10439F0F70180819181081B190BB8
:1023C000C80FD91FCC24DD2422C08091E80085FDF0
:1023D00016C08091E8008E778093E80037D1E11431
:1023E000F10449F0F701808191818C0D9D1D91834D
:1023F000808385E010C0BADD882349F00CC0899144
:102400008093F100015010400894C11CD11C0115AB
:102410001105D9F68B2DDF91CF911F910F91FF9070
:10242000EF90DF90CF90BF9008950F931F93DF93AD
:10243000CF9300D0CDB7DEB7EDE4F1E08091F100AD
:10244000819381E0E535F807C9F7FFD08091E80076
:1024500083FFE6C080914D0190914E01953009F4C3
:102460006DC0963040F4913081F1913070F093302E
:1024700009F0D6C02AC0983009F4A4C0993009F4F4
:10248000B3C0963009F0CCC07CC0803809F4C8C015
:10249000823809F0C5C0809151018F708093E900A6
:1024A0008091EB001092E9002091E800277F2093B3
:1024B000E80090E025E0969587952A95E1F78170F0
:1024C0008093F1001092F10088C0882319F08230C7
:1024D00009F0A6C08F71823009F0A2C080914F012F
:1024E000882331F5209151012F7009F499C0209370
:1024F000E9008091EB0080FF1BC0933021F48091B4
:10250000EB00806213C08091EB0080618093EB0050
:1025100081E090E002C0880F991F2A95E2F780932E
:10252000EA001092EA008091EB0088608093EB0053
:102530001092E9008091E800877F52C0882309F05B
:102540006FC010914F011F770FB7F8948091E8008A
:10255000877F8093E800EBDC8091E80080FFFCCF70
:102560008091E3008078812B8093E30080688093E2
:10257000E300112311F482E001C083E08EBB0FBFA2
:102580004FC08058823008F04BC080914F0190912D
:10259000500160915101AE014F5F5F4F0E94950164
:1025A000BC01009709F43CC08091E800877F8093CC
:1025B000E80089819A81EFDD8091E8008B77809334
:1025C000E8002EC0803861F58091E800877F809315
:1025D000E80080914B018093F1008091E8008E77B4
:1025E0008093E800A4DC1CC08823D1F490914F01B3
:1025F0009230B0F48091E800877F8093E800909358
:102600004B0195DC80914B01882331F48091E300EC
:1026100087FD02C081E001C084E08EBB0E945501AD
:102620008091E80083FF0AC08091EB008062809374
:10263000EB008091E800877F8093E8000F900F9077
:10264000CF91DF911F910F91089508951F938EB33D
:10265000882361F01091E9001092E9008091E80070
:1026600083FF01C0E2DE1F701093E9001F910895FF
:10267000F999FECF92BD81BDF89A992780B508954A
:10268000262FF999FECF92BD81BDF89A019700B42B
:10269000021639F01FBA20BD0FB6F894FA9AF99ACB
:0826A0000FBE0895F894FFCF6E
:1026A8004156524953505F4D4B3200800100810121
:1026B80000900100910101920111940121980306F3
:1026C8009E0301A10100A4030001C0010001200034
:1026D80033321289AB45CDD888FF1289AB45CDD8A6
:0226E80088FF69
:00000001FF
